:100000000C94620C0C948A0C0C948A0C0C948A0C40
:100010000C948A0C0C948A0C0C948A0C0C948A0C08
:100020000C948A0C0C948A0C0C948A0C0C948A0CF8
:100030000C948A0C0C948A0C0C948A0C0C948A0CE8
:100040000C94830D0C948A0C0C948A0C0C948A0CDE
:100050000C948A0C0C948A0C0C948A0C0C948A0CC8
:100060000C948A0C0C948A0C0000000023002600DB
:100070002900FFFFFFFFFFFFFFFFFFFFFFFFFFFF65
:10008000FFFFFFFFFFFFFFFFFFFFFFFFFFFFFFFF80
:10009000FFFFFFFFFFFFFFFFFFFFFFFFFFFFFFFF70
:1000A000FFFFFFFFFFFFFFFFFFFFFFFFFFFFFFFF60
:1000B000FFFFFFFFFFFFFFFFFFFFFFFFFFFFFFFF50
:10047000FFFF7F7F7E7E7E7E7D7D7D7D7C7C7C7CA4
:100480007B7B7B7B7A7A7A7A7979797978787878D4
:100490007777777776767676757575757474747404
:1004A0007373737372727272717171717070707034
:1004B0006F6F6F6F6E6E6E6E6D6D6D6D6C6C6C6C64
:1004C0006B6B6B6B6A6A6A6A696969696868686894
:1004D00067676767666666666565656564646464C4
:1004E00063636363626262626161616160606060F4
:1004F0005F5F5F5F5E5E5E5E5D5D5D5D5C5C5C5C24
:100500005B5B5B5B5A5A5A5A595959595858585853
:100510005757575756565656555555555554545482
:1005200054535353535252525251515151505050AF
:10053000504F4F4F4F4E4E4E4E4D4D4D4D4C4C4CDF
:100540004C4B4B4B4B4A4A4A4A494949494848480F
:10055000484747474746464646454545454444443F
:10056000444343434342424242414141414040406F
:10057000403F3F3F3F3E3E3E3E3D3D3D3D3C3C3C9F
:100580003C3B3B3B3B3A3A3A3A39393939383838CF
:1005900038373737373636363635353535343434FF
:1005A000343333333332323232313131313030302F
:1005B000302F2F2F2F2E2E2E2E2D2D2D2D2C2C2C5F
:1005C0002C2B2B2B2B2A2A2A2A292929292828288F
:1005D00028272727272626262625252525242424BF
:1005E00024232323232222222221212121202020EF
:1005F000201F1F1F1F1E1E1E1E1D1D1D1D1C1C1C1F
:100600001C1B1B1B1B1A1A1A1A191919191818184E
:10061000181717171716161616151515151414147E
:1006200014131313131212121211111111101010AE
:10063000100F0F0F0F0E0E0E0E0D0D0D0D0C0C0CDE
:100640000C0B0B0B0B0A0A0A0A090909090808080E
:10065000080707070706060606050505050404043E
:10066000040303030302020202010101010000006E
:100670000000FFFEFEFEFEFDFDFDFDFCFCFCFCFBA4
:10068000FBFBFBFAFAFAFAF9F9F9F9F8F8F8F8F7D6
:10069000F7F7F7F6F6F6F6F5F5F5F5F4F4F4F4F306
:1006A000F3F3F3F2F2F2F2F1F1F1F1F0F0F0F0EF36
:1006B000EFEFEFEEEEEEEEEDEDEDEDECECECECEB66
:1006C000EBEBEBEAEAEAEAE9E9E9E9E8E8E8E8E796
:1006D000E7E7E7E6E6E6E6E5E5E5E5E4E4E4E4E3C6
:1006E000E3E3E3E2E2E2E2E1E1E1E1E0E0E0E0DFF6
:1006F000DFDFDFDEDEDEDEDDDDDDDDDCDCDCDCDB26
:10070000DBDBDBDADADADAD9D9D9D9D8D8D8D8D755
:10071000D7D7D7D6D6D6D6D5D5D5D5D4D4D4D4D385
:10072000D3D3D3D2D2D2D2D1D1D1D1D0D0D0D0CFB5
:10073000CFCFCFCECECECECDCDCDCDCCCCCCCCCBE5
:10074000CBCBCBCACACACAC9C9C9C9C8C8C8C8C715
:10075000C7C7C7C6C6C6C6C5C5C5C5C4C4C4C4C345
:10076000C3C3C3C2C2C2C2C1C1C1C1C0C0C0C0BF75
:10077000BFBFBFBEBEBEBEBDBDBDBDBCBCBCBCBBA5
:10078000BBBBBBBABABABAB9B9B9B9B8B8B8B8B7D5
:10079000B7B7B7B6B6B6B6B5B5B5B5B4B4B4B4B305
:1007A000B3B3B3B2B2B2B2B1B1B1B1B0B0B0B0AF35
:1007B000AFAFAFAEAEAEAEADADADADACACACACAB65
:1007C000ABABABAAAAAAAAAAA9A9A9A9A8A8A8A892
:1007D000A7A7A7A7A6A6A6A6A5A5A5A5A4A4A4A4C1
:1007E000A3A3A3A3A2A2A2A2A1A1A1A1A0A0A0A0F1
:1007F0009F9F9F9F9E9E9E9E9D9D9D9D9C9C9C9C21
:100800009B9B9B9B9A9A9A9A999999999898989850
:100810009797979796969696959595959494949480
:1008200093939393929292929191919190909090B0
:100830008F8F8F8F8E8E8E8E8D8D8D8D8C8C8C8CE0
:100840008B8B8B8B8A8A8A8A898989898888888810
:100850008787878786868686858585858484848440
:100860008383838382828282818181818080808070
:100870007F7F7F7F80808080818181818282828270
:100880008383838384848484858585858686868620
:100890008787878788888888898989898A8A8A8AD0
:1008A0008B8B8B8B8C8C8C8C8D8D8D8D8E8E8E8E80
:1008B0008F8F8F8F90909090919191919292929230
:1008C00093939393949494949595959596969696E0
:1008D0009797979798989898999999999A9A9A9A90
:1008E0009B9B9B9B9C9C9C9C9D9D9D9D9E9E9E9E40
:1008F0009F9F9F9FA0A0A0A0A1A1A1A1A2A2A2A2F0
:10090000A3A3A3A3A4A4A4A4A5A5A5A5A6A6A6A69F
:10091000A7A7A7A7A8A8A8A8A9A9A9A9AAAAAAAA4F
:10092000AAABABABABACACACACADADADADAEAEAE03
:10093000AEAFAFAFAFB0B0B0B0B1B1B1B1B2B2B2B3
:10094000B2B3B3B3B3B4B4B4B4B5B5B5B5B6B6B663
:10095000B6B7B7B7B7B8B8B8B8B9B9B9B9BABABA13
:10096000BABBBBBBBBBCBCBCBCBDBDBDBDBEBEBEC3
:10097000BEBFBFBFBFC0C0C0C0C1C1C1C1C2C2C273
:10098000C2C3C3C3C3C4C4C4C4C5C5C5C5C6C6C623
:10099000C6C7C7C7C7C8C8C8C8C9C9C9C9CACACAD3
:1009A000CACBCBCBCBCCCCCCCCCDCDCDCDCECECE83
:1009B000CECFCFCFCFD0D0D0D0D1D1D1D1D2D2D233
:1009C000D2D3D3D3D3D4D4D4D4D5D5D5D5D6D6D6E3
:1009D000D6D7D7D7D7D8D8D8D8D9D9D9D9DADADA93
:1009E000DADBDBDBDBDCDCDCDCDDDDDDDDDEDEDE43
:1009F000DEDFDFDFDFE0E0E0E0E1E1E1E1E2E2E2F3
:100A0000E2E3E3E3E3E4E4E4E4E5E5E5E5E6E6E6A2
:100A1000E6E7E7E7E7E8E8E8E8E9E9E9E9EAEAEA52
:100A2000EAEBEBEBEBECECECECEDEDEDEDEEEEEE02
:100A3000EEEFEFEFEFF0F0F0F0F1F1F1F1F2F2F2B2
:100A4000F2F3F3F3F3F4F4F4F4F5F5F5F5F6F6F662
:100A5000F6F7F7F7F7F8F8F8F8F9F9F9F9FAFAFA12
:100A6000FAFBFBFBFBFCFCFCFCFDFDFDFDFEFEFEC2
:100A7000FEFF00000000000101010102020202036A
:100A8000030303040404040505050506060606071A
:100A900007070708080808090909090A0A0A0A0BCA
:100AA0000B0B0B0C0C0C0C0D0D0D0D0E0E0E0E0F7A
:100AB0000F0F0F101010101111111112121212132A
:100AC00013131314141414151515151616161617DA
:100AD00017171718181818191919191A1A1A1A1B8A
:100AE0001B1B1B1C1C1C1C1D1D1D1D1E1E1E1E1F3A
:100AF0001F1F1F20202020212121212222222223EA
:100B00002323232424242425252525262626262799
:100B100027272728282828292929292A2A2A2A2B49
:100B20002B2B2B2C2C2C2C2D2D2D2D2E2E2E2E2FF9
:100B30002F2F2F30303030313131313232323233A9
:100B40003333333434343435353535363636363759
:100B500037373738383838393939393A3A3A3A3B09
:100B60003B3B3B3C3C3C3C3D3D3D3D3E3E3E3E3FB9
:100B70003F3F3F4040404041414141424242424369
:100B80004343434444444445454545464646464719
:100B900047474748484848494949494A4A4A4A4BC9
:100BA0004B4B4B4C4C4C4C4D4D4D4D4E4E4E4E4F79
:100BB0004F4F4F5050505051515151525252525329
:100BC00053535354545454555555555556565656DB
:100BD0005757575758585858595959595A5A5A5A8D
:100BE0005B5B5B5B5C5C5C5C5D5D5D5D5E5E5E5E3D
:100BF0005F5F5F5F606060606161616162626262ED
:100C0000636363636464646465656565666666669C
:100C10006767676768686868696969696A6A6A6A4C
:100C20006B6B6B6B6C6C6C6C6D6D6D6D6E6E6E6EFC
:100C30006F6F6F6F707070707171717172727272AC
:100C4000737373737474747475757575767676765C
:100C50007777777778787878797979797A7A7A7A0C
:100C60007B7B7B7B7C7C7C7C7D7D7D7D7E7E7E7EBC
:100C70007F7FFFFFFFFFFFFFFFFFFFFFFFFFFFFF84
:100C8000FFFFFFFFFFFFFFFFFFFFFFFFFFFFFFFF74
:100C9000FFFFFFFFFFFFFFFFFFFFFFFFFFFFFFFF64
:100CA000FFFFFFFFFFFFFFFFFFFFFFFFFFFFFFFF54
:100CB000FFFFFFFFFFFFFFFFFFFFFFFFFFFFFFFF44
:100CC000FFFFFFFFFFFFFFFFFFFFFFFFFFFFFFFF34
:100CD000FFFFFFFFFFFFFFFFFFFFFFFFFFFFFFFF24
:100CE000FFFFFFFFFFFFFFFFFFFFFFFFFFFFFFFF14
:100CF000FFFFFFFFFFFFFFFFFFFFFFFFFFFFFFFF04
:100D0000FFFFFFFFFFFFFFFFFFFFFFFFFFFFFFFFF3
:100D1000FFFFFFFFFFFFFFFFFFFFFFFFFFFFFFFFE3
:100D2000FFFFFFFFFFFFFFFFFFFFFFFFFFFFFFFFD3
:100D3000FFFFFFFFFFFFFFFFFFFFFFFFFFFFFFFFC3
:100D4000FFFFFFFFFFFFFFFFFFFFFFFFFFFFFFFFB3
:100D5000FFFFFFFFFFFFFFFFFFFFFFFFFFFFFFFFA3
:100D6000FFFFFFFFFFFFFFFFFFFFFFFFFFFFFFFF93
:100D7000FFFFFFFFFFFFFFFFFFFFFFFFFFFFFFFF83
:100D8000FFFFFFFFFFFFFFFFFFFFFFFFFFFFFFFF73
:100D9000FFFFFFFFFFFFFFFFFFFFFFFFFFFFFFFF63
:100DA000FFFFFFFFFFFFFFFFFFFFFFFFFFFFFFFF53
:100DB000FFFFFFFFFFFFFFFFFFFFFFFFFFFFFFFF43
:100DC000FFFFFFFFFFFFFFFFFFFFFFFFFFFFFFFF33
:100DD000FFFFFFFFFFFFFFFFFFFFFFFFFFFFFFFF23
:100DE000FFFFFFFFFFFFFFFFFFFFFFFFFFFFFFFF13
:100DF000FFFFFFFFFFFFFFFFFFFFFFFFFFFFFFFF03
:100E0000FFFFFFFFFFFFFFFFFFFFFFFFFFFFFFFFF2
:100E1000FFFFFFFFFFFFFFFFFFFFFFFFFFFFFFFFE2
:100E2000FFFFFFFFFFFFFFFFFFFFFFFFFFFFFFFFD2
:100E3000FFFFFFFFFFFFFFFFFFFFFFFFFFFFFFFFC2
:100E4000FFFFFFFFFFFFFFFFFFFFFFFFFFFFFFFFB2
:100E5000FFFFFFFFFFFFFFFFFFFFFFFFFFFFFFFFA2
:100E6000FFFFFFFFFFFFFFFFFFFFFFFFFFFFFFFF92
:100E7000FFFF000000000000000000000000000074
:100E80000000000000000000000000000000000062
:100E90000000000000000000000000000000000052
:100EA0000000000000000000000000000000000042
:100EB0000000000000000000000000000000000032
:100EC0000000000000000000000000000000000022
:100ED0000000000000000000000000000000000012
:100EE0000000000000000000000000000000000002
:100EF00000000000000000000000000000000000F2
:100F000000000000000000000000000000000000E1
:100F100000000000000000000000000000000000D1
:100F200000000000000000000000000000000000C1
:100F300000000000000000000000000000000000B1
:100F400000000000000000000000000000000000A1
:100F50000000000000000000000000000000000091
:100F60000000000000000000000000000000000081
:100F70000000000000000000000000000000000071
:100F80000000000000000000000000000000000061
:100F90000000000000000000000000000000000051
:100FA0000000000000000000000000000000000041
:100FB0000000000000000000000000000000000031
:100FC0000000000000000000000000000000000021
:100FD0000000000000000000000000000000000011
:100FE0000000000000000000000000000000000001
:100FF00000000000000000000000000000000000F1
:1010000000000000000000000000000000000000E0
:1010100000000000000000000000000000000000D0
:1010200000000000000000000000000000000000C0
:1010300000000000000000000000000000000000B0
:1010400000000000000000000000000000000000A0
:101050000000000000000000000000000000000090
:101060000000000000000000000000000000000080
:10107000000000000001010202030304040505064C
:10108000060707080809090A0A0B0B0C0C0D0D0EC0
:101090000E0F0F1010111112121313141415151630
:1010A000161717181819191A1A1B1B1C1C1D1D1EA0
:1010B0001E1F1F2020212122222323242425252610
:1010C000262727282829292A2A2B2B2C2C2D2D2E80
:1010D0002E2F2F30303131323233333434353536F0
:1010E000363737383839393A3A3B3B3C3C3D3D3E60
:1010F0003E3F3F40404141424243434444454546D0
:10110000464747484849494A4A4B4B4C4C4D4D4E3F
:101110004E4F4F50505151525253535454555556AF
:10112000565757585859595A5A5B5B5C5C5D5D5E1F
:101130005E5F5F606061616262636364646565668F
:10114000666767686869696A6A6B6B6C6C6D6D6EFF
:101150006E6F6F707071717272737374747575766F
:10116000767777787879797A7A7B7B7C7C7D7D7EDF
:101170007E7F7F7F80808181828283838484858556
:1011800086868787888889898A8A8B8B8C8C8D8DC7
:101190008E8E8F8F90909191929293939494959537
:1011A00096969797989899999A9A9B9B9C9C9D9DA7
:1011B0009E9E9F9FA0A0A1A1A2A2A3A3A4A4A5A517
:1011C000A6A6A7A7A8A8A9A9AAAAABABACACADAD87
:1011D000AEAEAFAFB0B0B1B1B2B2B3B3B4B4B5B5F7
:1011E000B6B6B7B7B8B8B9B9BABABBBBBCBCBDBD67
:1011F000BEBEBFBFC0C0C1C1C2C2C3C3C4C4C5C5D7
:10120000C6C6C7C7C8C8C9C9CACACBCBCCCCCDCD46
:10121000CECECFCFD0D0D1D1D2D2D3D3D4D4D5D5B6
:10122000D6D6D7D7D8D8D9D9DADADBDBDCDCDDDD26
:10123000DEDEDFDFE0E0E1E1E2E2E3E3E4E4E5E596
:10124000E6E6E7E7E8E8E9E9EAEAEBEBECECEDED06
:10125000EEEEEFEFF0F0F1F1F2F2F3F3F4F4F5F576
:10126000F6F6F7F7F8F8F9F9FAFAFBFBFCFCFDFDE6
:10127000FEFEFFFEFEFDFDFCFCFBFBFAFAF9F9F8B1
:10128000F8F7F7F6F6F5F5F4F4F3F3F2F2F1F1F01E
:10129000F0EFEFEEEEEDEDECECEBEBEAEAE9E9E88E
:1012A000E8E7E7E6E6E5E5E4E4E3E3E2E2E1E1E0FE
:1012B000E0DFDFDEDEDDDDDCDCDBDBDADAD9D9D86E
:1012C000D8D7D7D6D6D5D5D4D4D3D3D2D2D1D1D0DE
:1012D000D0CFCFCECECDCDCCCCCBCBCACAC9C9C84E
:1012E000C8C7C7C6C6C5C5C4C4C3C3C2C2C1C1C0BE
:1012F000C0BFBFBEBEBDBDBCBCBBBBBABAB9B9B82E
:10130000B8B7B7B6B6B5B5B4B4B3B3B2B2B1B1B09D
:10131000B0AFAFAEAEADADACACABABAAAAA9A9A80D
:10132000A8A7A7A6A6A5A5A4A4A3A3A2A2A1A1A07D
:10133000A09F9F9E9E9D9D9C9C9B9B9A9A999998ED
:10134000989797969695959494939392929191905D
:10135000908F8F8E8E8D8D8C8C8B8B8A8A898988CD
:10136000888787868685858484838382828181803D
:10137000807F7F7F7E7E7D7D7C7C7B7B7A7A7979A6
:101380007878777776767575747473737272717115
:1013900070706F6F6E6E6D6D6C6C6B6B6A6A696985
:1013A00068686767666665656464636362626161F5
:1013B00060605F5F5E5E5D5D5C5C5B5B5A5A595965
:1013C00058585757565655555454535352525151D5
:1013D00050504F4F4E4E4D4D4C4C4B4B4A4A494945
:1013E00048484747464645454444434342424141B5
:1013F00040403F3F3E3E3D3D3C3C3B3B3A3A393925
:101400003838373736363535343433333232313194
:1014100030302F2F2E2E2D2D2C2C2B2B2A2A292904
:101420002828272726262525242423232222212174
:1014300020201F1F1E1E1D1D1C1C1B1B1A1A1919E4
:101440001818171716161515141413131212111154
:1014500010100F0F0E0E0D0D0C0C0B0B0A0A0909C4
:101460000808070706060505040403030202010134
:1014700000007F8081818283848485868788888933
:101480008A8B8B8C8D8E8F8F909192929394959660
:1014900096979899999A9B9C9C9D9E9F9FA0A1A28C
:1014A000A3A3A4A5A6A6A7A8A8A9AAABABACADAEBA
:1014B000AEAFB0B1B1B2B3B3B4B5B6B6B7B8B8B9F0
:1014C000BABABBBCBCBDBEBFBFC0C1C1C2C3C3C42E
:1014D000C5C5C6C6C7C8C8C9CACACBCCCCCDCDCE77
:1014E000CFCFD0D0D1D2D2D3D3D4D5D5D6D6D7D7CB
:1014F000D8D9D9DADADBDBDCDCDDDDDEDFDFE0E02A
:10150000E1E1E2E2E3E3E4E4E4E5E5E6E6E7E7E897
:10151000E8E9E9E9EAEAEBEBECECECEDEDEEEEEE16
:10152000EFEFEFF0F0F1F1F1F2F2F2F3F3F3F4F4A4
:10153000F4F4F5F5F5F6F6F6F7F7F7F7F8F8F8F846
:10154000F9F9F9F9F9FAFAFAFAFAFBFBFBFBFBFCF9
:10155000FCFCFCFCFCFCFDFDFDFDFDFDFDFDFEFEBF
:10156000FEFEFEFEFEFEFEFEFEFEFEFEFEFEFEFE9B
:10157000FEFEFFFEFEFEFEFEFEFEFEFEFEFEFEFE8A
:10158000FEFEFEFEFEFEFEFDFDFDFDFDFDFDFDFC85
:10159000FCFCFCFCFCFCFBFBFBFBFBFAFAFAFAFA9A
:1015A000F9F9F9F9F9F8F8F8F8F7F7F7F7F6F6F6C0
:1015B000F5F5F5F4F4F4F4F3F3F3F2F2F2F1F1F1FA
:1015C000F0F0EFEFEFEEEEEEEDEDECECECEBEBEA46
:1015D000EAE9E9E9E8E8E7E7E6E6E5E5E4E4E4E3A3
:1015E000E3E2E2E1E1E0E0DFDFDEDDDDDCDCDBDB0E
:1015F000DADAD9D9D8D7D7D6D6D5D5D4D3D3D2D28B
:10160000D1D0D0CFCFCECDCDCCCCCBCACAC9C8C813
:10161000C7C6C6C5C5C4C3C3C2C1C1C0BFBFBEBDA6
:10162000BCBCBBBABAB9B8B8B7B6B6B5B4B3B3B246
:10163000B1B1B0AFAEAEADACABABAAA9A8A8A7A6EE
:10164000A6A5A4A3A3A2A1A09F9F9E9D9C9C9B9A9C
:10165000999998979696959493929291908F8F8E50
:101660008D8C8B8B8A898888878685848483828108
:1016700081807F7E7D7D7C7B7A7A797877767675BE
:101680007473737271706F6F6E6D6C6C6B6A696876
:1016900068676665656463626261605F5F5E5D5C2A
:1016A0005B5B5A59585857565655545353525150DC
:1016B000504F4E4D4D4C4B4B4A4948484746464586
:1016C000444443424241403F3F3E3D3D3C3B3B3A28
:1016D00039393838373636353434333232313130BF
:1016E0002F2F2E2E2D2C2C2B2B2A2929282827274B
:1016F0002625252424232322222121201F1F1E1ECC
:101700001D1D1C1C1B1B1A1A1A191918181717163D
:10171000161515151414131312121211111010109E
:101720000F0F0F0E0E0D0D0D0C0C0C0B0B0B0A0AF0
:101730000A0A09090908080807070707060606062E
:10174000050505050504040404040303030303025B
:101750000202020202020101010101010101000075
:101760000000000000000000000000000000000079
:101770000000000000000000000000000000000069
:10178000000000000000000101010101010101024F
:10179000020202020202030303030304040404041A
:1017A00005050505050606060607070707080808D4
:1017B0000909090A0A0A0A0B0B0B0C0C0C0D0D0D7A
:1017C0000E0E0F0F0F10101011111212121313140E
:1017D0001415151516161717181819191A1A1A1B91
:1017E0001B1C1C1D1D1E1E1F1F2021212222232306
:1017F00024242525262727282829292A2B2B2C2C69
:101800002D2E2E2F2F3031313232333434353636BF
:1018100037383839393A3B3B3C3D3D3E3F3F40410C
:101820004242434444454646474848494A4B4B4C4C
:101830004D4D4E4F50505152535354555656575884
:1018400058595A5B5B5C5D5E5F5F606162626364B6
:10185000656566676868696A6B6C6C6D6E6F6F70E2
:1018600071727373747576767778797A7A7B7C7D0A
:101870007D7E00000000240027002A0000000000F8
:10188000250028002B0004040404040404040202BC
:1018900002020202030303030303010204081020EF
:1018A00040800102040810200102040810200000FA
:1018B000000800020100000304070000000000000F
:1018C00000000C1011241FBECFEFD8E0DEBFCDBF4B
:1018D00011E0A0E0B1E0EAE5F4E202C005900D926B
:1018E000A830B107D9F721E0A8E0B1E001C01D920E
:1018F000AF32B207E1F71CE0C2E6DCE004C021979A
:10190000FE010E942512C136D107C9F70E94CD0DF4
:101910000C942B120C940000833081F028F4813059
:1019200099F08230A9F008958730A9F08830C9F085
:101930008430B1F4809180008F7D03C0809180005D
:101940008F7780938000089584B58F7784BD089544
:1019500084B58F7DFBCF8091B0008F778093B000EE
:1019600008958091B0008F7DF9CF1F93CF93DF93BF
:10197000282F30E0F901E255F74E8491F901E6563F
:10198000F74ED491F901EA57F74EC491CC23A9F050
:10199000162F81110E948C0CEC2FF0E0EE0FFF1F30
:1019A000E458F74EA591B4918FB7F894EC911111CA
:1019B00008C0D095DE23DC938FBFDF91CF911F91BC
:1019C0000895DE2BF8CFCF93DF9390E0FC01E6562D
:1019D000F74E24918A57974EFC0184918823D1F0C9
:1019E00090E0880F991FFC01EE58F74EA591B49135
:1019F000FC01E458F74EC591D491623071F49FB761
:101A0000F8943C91822F809583238C93E8812E2B30
:101A100028839FBFDF91CF9108958FB7F894EC9101
:101A20002E2B2C938FBFF6CF1F93CF93DF93182FBE
:101A3000EB0161E00E94E30C209739F460E0812F14
:101A4000DF91CF911F910C94B50CCF3FD10511F4CC
:101A500061E0F5CFE12FF0E0E255F74EE491E3309D
:101A600031F140F4E130B1F0E230E1F0C038D105BD
:101A70007CF7E4CFE73029F1E83059F1E430B1F7F1
:101A800080918000806280938000D0938B00C0930F
:101A90008A0004C084B5806884BDC7BDDF91CF9142
:101AA0001F91089584B5806284BDC8BDF7CF809131
:101AB0008000806880938000D0938900C093880064
:101AC000EDCF8091B00080688093B000C093B300E8
:101AD000E5CF8091B00080628093B000C093B400E5
:101AE000DDCF8E50806480937C0080917A0080648A
:101AF00080937A0080917A0086FDFCCF80917800F7
:101B00009091790008951F920F920FB60F921124B1
:101B10002F933F938F939F93AF93BF9380912B010C
:101B200090912C01A0912D01B0912E0130912A01AC
:101B300023E0230F2D3758F50196A11DB11D2093E9
:101B40002A0180932B0190932C01A0932D01B09337
:101B50002E018091260190912701A0912801B0913A
:101B600029010196A11DB11D8093260190932701A3
:101B7000A0932801B0932901BF91AF919F918F91BC
:101B80003F912F910F900FBE0F901F90189526E850
:101B9000230F0296A11DB11DD2CF789484B5826027
:101BA00084BD84B5816084BD85B5826085BD85B501
:101BB000816085BD80916E00816080936E0010927F
:101BC00081008091810082608093810080918100FA
:101BD000816080938100809180008160809380008B
:101BE0008091B10084608093B1008091B0008160E9
:101BF0008093B00080917A00846080937A00809115
:101C00007A00826080937A0080917A00816080936C
:101C10007A0080917A00806880937A001092C100E7
:101C200062E084E00E94E30C61E083E00E94E30C48
:101C300061E08BE00E94E30C90E080E00E942010C5
:101C400090E0909307018093060183E28093B000B7
:101C500081E08093B10082E88093800089E18093E5
:101C600081008FEF90E090938700809386004AE890
:101C7000242E48E1342EEE24EA94F12C60E0C62EA6
:101C800060E0D62E8FB7F89480902B0190902C01B5
:101C9000A0902D01B0902E018FBF809222019092D2
:101CA0002301A0922401B0922501E2EBF8E1849196
:101CB000EEE9F8E1C491F101D491DD2379F08111CD
:101CC0000E948C0CED2FF0E0EE0FFF1FE859FF4F44
:101CD000A591B4918C91C82381E009F480E0109221
:101CE00020011092210190911F01891751F08093DA
:101CF0001F0180921A0190921B01A0921C01B092C8
:101D00001D0180911A0190911B01A0911C01B091BD
:101D10001D01881A990AAA0ABB0A8091160190919E
:101D20001701A0911801B091190188159905AA050C
:101D3000BB05B0F490911E0180911F01981781F0AE
:101D400080931E01911103C021E0813009F020E051
:101D500020932001913009F4811190E090932101AA
:101D600080912101882381F08091060190910701E3
:101D70006AE0019709F061E06093060110920701A3
:101D800090E080E00E9428108EE00E94710DEC012E
:101D900081E10E94710DAC01CE01DD0FAA0BBB0BDE
:101DA000052E000C660B770B840F951FA61FB71F1F
:101DB000B7FD0FC18115F4E09F07A105B1050CF037
:101DC0000BC1BC01990F880B990B0E94DB1026EA0E
:101DD0003BE944EC5AE30E946C114B015C016091B9
:101DE000060170910701072E000C880B990B0E94C9
:101DF000DB109B01AC01C501B4010E946C114B01C9
:101E00005C018092020190920301A0920401B092C1
:101E100005018FE00E94710D8C0182E10E94710D1D
:101E2000012E000C220B330B092E000CAA0BBB0B4E
:101E3000800F911FA21FB31F10E000E0B7FD08C084
:101E40008C0181159440A105B10514F00FEF13E04A
:101E5000109315010093140180E10E94710D782EFA
:101E6000D92F83E10E94710D272D3D2F37FF02C02E
:101E70002D5F3F4FE901D595C795D595C7959C0135
:101E800097FF02C02D5F3F4F3595279535952795D4
:101E9000C20FD31FCF3FD10519F014F0CFEFD0E020
:101EA000D0930101C0930001809122019091230100
:101EB000A0912401B0912501409110015091110190
:101EC000609112017091130184179507A607B70757
:101ED00009F478C08093100190931101A09312012E
:101EE000B093130140900C0150900D0160900E01D1
:101EF00070900F01C301B2010E94A310FB01EE58C4
:101F0000FB4E07361105C4F00533E1E01E070CF463
:101F10006EC00330F2E01F070CF465C0FB01EE5801
:101F2000F74F013D22E012073CF00F3913400CF44B
:101F300056C0FB01EE58FF4FE491EC9FC001ED9FAE
:101F4000900D1124B7010E94FD11CB01770FAA0B50
:101F5000BB0B8093080190930901A0930A01B093F1
:101F60000B0180910801C82F70910901682F8BE047
:101F70000E94140DF0E4CF9FC0011124B7010E940C
:101F8000FD1183E00E94140DA5019401C301B2016B
:101F90000E9437102AE037ED43E25CE30E943710DD
:101FA0004B015C0120E030E040E854E40E946711FE
:101FB00087FF21C080920C0190920D01A0920E012A
:101FC000B0920F01C114D10409F45CCE0E9400004C
:101FD00059CE90E080E0F5CE8FEF93E0F2CEFB019A
:101FE000EE58FB4FA9CFFB01EE58F34FA5CFFB01F5
:101FF000EE58FF4EA1CF20E030E040E854E4C501A8
:10200000B4010E94361060930C0170930D0180930F
:102010000E0190930F01D6CFE6E1F1E082E390E06C
:10202000A0E0B0E080839183A283B3831482158201
:102030001682178281E08087818712861386089531
:10204000F999FECF92BD81BDF89A992780B5089580
:10205000262FF999FECF1FBA92BD81BD20BD0FB6C4
:10206000F894FA9AF99A0FBE019608955058BB2732
:10207000AA270E944E100C942D110E941F1138F0B7
:102080000E94261120F039F49F3F19F426F40C9495
:102090001C110EF4E095E7FB0C941611E92F0E9439
:1020A0003E1158F3BA17620773078407950720F0AB
:1020B00079F4A6F50C9460110EF4E0950B2EBA2F6E
:1020C000A02D0B01B90190010C01CA01A00111243E
:1020D000FF27591B99F0593F50F4503E68F11A16EA
:1020E000F040A22F232F342F4427585FF3CF46957B
:1020F00037952795A795F0405395C9F77EF41F169D
:10210000BA0B620B730B840BBAF09150A1F0FF0F66
:10211000BB1F661F771F881FC2F70EC0BA0F621F52
:10212000731F841F48F4879577956795B795F79542
:102130009E3F08F0B0CF9395880F08F09927EE0FD7
:102140009795879508950E94AA106894B1110C94F0
:10215000611108950E94461188F09F5798F0B92F99
:102160009927B751B0F0E1F0660F771F881F991FCC
:102170001AF0BA95C9F714C0B13091F00E946011FD
:10218000B1E008950C946011672F782F8827B85F0D
:1021900039F0B93FCCF3869577956795B395D9F724
:1021A0003EF490958095709561957F4F8F4F9F4F2E
:1021B0000895E89409C097FB3EF49095809570953A
:1021C00061957F4F8F4F9F4F9923A9F0F92F96E983
:1021D000BB279395F695879577956795B795F111F8
:1021E000F8CFFAF4BB0F11F460FF1BC06F5F7F4F95
:1021F0008F4F9F4F16C0882311F096E911C07723A7
:1022000021F09EE8872F762F05C0662371F096E8AF
:10221000862F70E060E02AF09A95660F771F881F7E
:10222000DAF7880F9695879597F9089597F99F673C
:1022300080E870E060E008959FEF80EC089500244E
:102240000A941616170618060906089500240A941B
:1022500012161306140605060895092E0394000CA1
:1022600011F4882352F0BB0F40F4BF2B11F460FF30
:1022700004C06F5F7F4F8F4F9F4F089557FD905859
:10228000440F551F59F05F3F71F04795880F97FB3A
:10229000991F61F09F3F79F08795089512161306F4
:1022A0001406551FF2CF4695F1DF08C01616170623
:1022B0001806991FF1CF8695710561050894089558
:1022C000E894BB2766277727CB0197F908950E94EA
:1022D000D91108F48FEF08950E947F110C942D11ED
:1022E0000E941F1138F00E94261120F0952311F052
:1022F0000C9416110C941C1111240C9461110E9461
:102300003E1170F3959FC1F3950F50E0551F629FEA
:10231000F001729FBB27F00DB11D639FAA27F00D3E
:10232000B11DAA1F649F6627B00DA11D661F829F65
:102330002227B00DA11D621F739FB00DA11D621F4A
:10234000839FA00D611D221F749F3327A00D611D67
:10235000231F849F600D211D822F762F6A2F112449
:102360009F5750409AF0F1F088234AF0EE0FFF1F7C
:10237000BB1F661F771F881F91505040A9F79E3FD3
:10238000510580F00C9416110C9461115F3FE4F339
:10239000983ED4F3869577956795B795F795E79529
:1023A0009F5FC1F7FE2B880F911D9695879597F932
:1023B0000895990F0008550FAA0BE0E8FEEF1616D6
:1023C0001706E807F907C0F012161306E407F50729
:1023D00098F0621B730B840B950B39F40A2661F09D
:1023E000232B242B252B21F408950A2609F4A14040
:1023F000A6958FEF811D811D089597FB072E16F47A
:10240000009407D077FD09D00E94111207FC05D077
:102410003EF4909581959F4F0895709561957F4FFB
:102420000895AA1BBB1B51E107C0AA1FBB1FA6171B
:10243000B70710F0A61BB70B881F991F5A95A9F76D
:1024400080959095BC01CD010895EE0FFF1F05907A
:0A245000F491E02D0994F894FFCFF9
:08245A00FF00CDCCCC3D0100D8
:00000001FF
